:103D34000ECF0EBB0EA70E920E7C0E650E4D0E34EA
:103D44000E190DFE0DE10DC40DA50D850D640D427A
:103D54000D1E0CFA0CD40CAE0C860C5D0C330C0846
:103D64000BDC0BB00B820B540B250AF50AC40A9327
:103D74000A610A2F09FD09CA09960963092F08FC7B
:103D840008C808950861082E07FB07C8079607644A
:103D94000733070206D206A206730645061705EA8C
:103DA40005BF059305690540051704F004C904A37C
:103DB400047E045A0437041503F403D303B40396AE
:103DC4000378035B033F0324030A02F002D702BF14
:103DD40002A80292027C02670253023F022C021ADA
:103DE400020801F701E601D601C701B801A9019C47
:103DF400018E018101740168015D01510146013C9C
:103E040001320128011F0115010D010400FC00F419
:103E140000EC00E500DE00D700D000CA00C300BDFE
:103E240000B800B200AD00A700A2009E0099009463
:103E34000090008C008700840080007C007800756E
:103E44000072006E006B0068006500620060005D37
:103E5400005A0058005500530051004E004C004ACF
:103E640000480046004400430041003F003E003C3F
:103E7400003A003900370036003500330032003193
:103E8400002F002E002D002C002B002A00290028D2
:103E94000027002600250024002300010C01010452
:103EA40002011E030A960401320502020600640799
:103EB400010108000009015A0E01010F000112005E
:103EC4006413010114013C1501FA1664FA17FFFF8B
:103ED4001D00072000072400022701012F013C30A8
:103EE400010132010335FFFF3603073CFFFF3DFFAD
:103EF400FF180002191E461A00021B00022D32C8C8
:103F04002E0001FAFAFA18000019FFFF1A00001B2C
:103F140000002D32C82E0001FAFAFA18000019FF29
:103F2400FF1A00001B00002DFFFF2EFFFFFAFAFA14
:10004800900786E0FEA3E0FF7457BE0010D39F40E0
:100058000C903E9E12001EE493F599804C9000147B
:10006800E0D394044014900786E0FEA3E0FF903E9E
:100078009E12001EE493F599802F900014E0D3940B
:10008800034014900786E0FEA3E0FF903EB3120001
:100098001EE493F5998012900786E0FEA3E0FF9096
:1000A8003EC812001EE493F59990078612000E9040
:1000B8000786E0FEA3E0FF746C6F4E7003751300B3
:1000C8002290013AE090002AF090013BE090002B4A
:1000D800F090013CE090002CF0A20AB34016900189
:1000E8003AE0700C90013BE0700690013CE0600241
:1000F8008002C20A90013AE0B4300F90013BE0B4AC
:10010800470890013CE0643B60028004D20B800207
:10011800C20BE558B40102800302023C900057E08C
:10012800F566900062E0F568900063E0F56990007C
:1001380074E0F56A90007AE0900029F090007CE085
:10014800F56590007DE0F567900080E0F56490002B
:1001580081E0F563900090E0900041F0900091E01C
:10016800900042F0900092E0900043F0900093E0FD
:10017800900044F0900094E0900045F0900095E0E5
:10018800900046F0900096E0900047F0900097E0CD
:10019800900048F0900099E0900033F090009AE0C9
:1001A800900034F090009BE0900035F090009CE0C7
:1001B800900036F0900079E0B4011790000A740FAF
:1001C800F0A374FFF090000CE4F0A3F07402900028
:1001D80079F0900079E0B4035990000CE0FEA3E0B8
:1001E800FF90000AE0FCA3E0FD1200037410124027
:1001F800947408124086EF900026F0EF700674FFA2
:10020800900026F07400900079F090000BE09000C8
:1002180027F090000AE0900028F0900026E0900770
:1002280089F0900027E090078AF0900028E0900776
:100238008BF0803F900081E070067558017563006F
:10024800A20AB3402E90013AE090002AF090013BB8
:10025800E090002BF090013CE090002CF090002AF8
:10026800E0700C90002BE0700690002CE06002809B
:1002780002C20AE5667003756602E5687003756870
:10028800027E837FC2E5668E048F05FF1240768C5E
:10029800398D3AE56975F0FAA4FFAEF0E5688E0489
:1002A8008F05FF1240768C3D8D3E90004FE0F56043
:1002B80090004DE0FE900069E0B5061890004CE013
:1002C800FE900068E0B5060C90004BE0FE900059E7
:1002D800E06E606F900069E07006900068E060066C
:1002E8007400900059F0900069E0B4020890004949
:1002F8007401F08005900049E4F0900068E0B402D1
:100308000890004A7401F0800590004AE4F09000DB
:1003180068E0600690004AE060028005756003802E
:1003280003756004E559B55802D20C900068E09056
:10033800004CF0900069E090004DF0900059E0907A
:10034800004BF0740190009EF0740090009FF074D0
:10035800009000A0F074009000A1F074009000A23A
:10036800F074009000A3F074009000A4F074019061
:1003780000A5F074009000A6F074009000A7F07437
:10038800009000A8F074009000A9F074009000AAF2
:10039800F074009000ABF074019000ACF074009021
:1003A80000ADF074009000AEF074009000AFF074EF
:1003B800009000B0F074009000B1F074009000B2AA
:1003C800F07401900362F07400900363F07400907D
:1003D8000364F07400900365F07400900366F07491
:1003E80000900367F07400900368F074019003A212
:1003F800F074019003A3F074009003A4F0740090CB
:1004080003A5F074009003A6F074009003A7F0749D
:10041800009003A8F074009003E2F074019003E3E5
:10042800F074009003E4F074009003E5F074009019
:1004380003E6F074009003E7F074009003E8F074AA
:1004480000900422F07400900423F07400900424B7
:10045800F07400900425F07400900426F074009065
:100468000427F07400900428F022E5B554F7F5B598
:10047800E5B554FDF5B5C2A2C2A1C292C207E5B561
:1004880054FBF5B5755104E55104F55290004FE061
:10049800F560900025E4F0C209E5B554FEF5B5C253
:1004A8008E758D00758B00754C00752600752500BE
:1004B800D28E22750A00750900AE09AF0A7457BEBC
:1004C80000039F5003020578903E9E12001EE4939D
:1004D80090004E1240AC0FBF00010EE0FC903E9E13
:1004E80012001EECFEE493FFEEC39F5026AE09AF48
:1004F8000A0FBF00010E903E9E12001EAE09AF0A01
:10050800E493FC903E9E12001EE49390004E12402D
:10051800ACECF0AE09AF0A903E9E12001EE4939038
:10052800004E1240ACE0FC903EA012001EECFCE431
:1005380093FDECD39D4019903EA012001EE493FC5D
:10054800903E9E12001EE49390004E1240ACECF0D8
:10055800AE09AF0A74022FFF50010E8E098F0A7878
:100568000A740126F6500418E436F640030204C162
:1005780022750A00750900AE09AF0A7415BE00039A
:100588009F5003020646903EF512001EE493900029
:100598004E1240AC0FBF00010EE0FC903EF5120079
:1005A8001EECFEE493FFEEC39F5026AE09AF0A0F80
:1005B800BF00010E903EF512001EAE09AF0AE4938B
:1005C800FC903EF512001EE49390004E1240ACECF5
:1005D800F0AE09AF0A903EF512001EE49390004E6B
:1005E8001240ACE0FC903EF712001EECFCE493FDD8
:1005F800ECD39D4019903EF712001EE493FC903E08
:10060800F512001EE49390004E1240ACECF0AE09D7
:10061800AF0A740F6F4E7006750A15750900AE099A
:10062800AF0A74022FFF50010E8E098F0A780A74E0
:100638000126F6500418E436F6400302057F2275B9
:100648000A00750900AE09AF0A7415BE00039F5071
:1006580003020714903F0A12001EE49390004E1202
:1006680040AC0FBF00010EE0FC903F0A12001EECE8
:10067800FEE493FFEEC39F5026AE09AF0A0FBF00FA
:10068800010E903F0A12001EAE09AF0AE493FC90D7
:100698003F0A12001EE49390004E1240ACECF0AEFC
:1006A80009AF0A903F0A12001EE49390004E1240D0
:1006B800ACE0FC903F0C12001EECFCE493FDECD384
:1006C8009D4019903F0C12001EE493FC903F0A12C3
:1006D800001EE49390004E1240ACECF0AE09AF0A55
:1006E800740F6F4E7006750A15750900AE09AF0ACA
:1006F80074022FFF50010E8E098F0A780A740126A2
:10070800F6500418E436F6400302064D22750A0036
:10071800750900AE09AF0A7415BE00039F500302A5
:1007280007E2903F1F12001EE49390004E1240AC67
:100738000FBF00010EE0FC903F1F12001EECFEE40C
:1007480093FFEEC39F5026AE09AF0A0FBF00010EFC
:10075800903F1F12001EAE09AF0AE493FC903F1FA2
:1007680012001EE49390004E1240ACECF0AE09AFBC
:100778000A903F1F12001EE49390004E1240ACE016
:10078800FC903F2112001EECFCE493FDECD39D404D
:1007980019903F2112001EE493FC903F1F12001E87
:1007A800E49390004E1240ACECF0AE09AF0A740F1F
:1007B8006F4E7006750A15750900AE09AF0A740206
:1007C8002FFF50010E8E098F0A780A740126F65001
:1007D8000418E436F6400302071B22054D22054C97
:1007E80022054EC2CF2290F800E49364066002808E
:1007F800FE75840175A70075FF80900788E4F07581
:10080800C91075A70F75A1C775A70075D90075CE52
:10081800FF75A70F75F1FE75F2FF75F33775F4785C
:1008280075A4BA75A5FF75A60775AE0075AFFF75F7
:10083800D48175D5FF75D6FF75D7FFC296C295C20C
:10084800A0C297E5B554BFF5B5E5B554DFF5B5E5F4
:10085800B554EFF5B5E5B5547FF5B5E5B554F7F5FD
:10086800B5E5B554FDF5B575A70075A20175A147A5
:1008780075F80975BC0175BE0475BD6C75BE077544
:10088800BDA075BE0875BD0175BC0075BB1875BCEB
:100898002075BA0875E88075D11375A70F75E1053D
:1008A80075E20075C740759700759780740A124005
:1008B800667597C0E5975420700280F8758F0275A9
:1008C800A700D2AF75980075A90C75A70F75AB4333
:1008D80075ADFB75AC1E75A700758911758E007511
:1008E8008C00758A00D2A9D28C758D00758B00D2C8
:1008F800ABD28E75CD0075CC0075CA0075CB00D211
:10090800ADC2CFD2CA7591047592007593CD75EFBB
:100918000675D94075CF01900786E4F0A3F07513EA
:1009280000751400C299D20AC20D12047274C8F577
:100938001875170012266375A70FE5FB90001AF0CB
:10094800E5FA90001BF0E5F990001CF075A70090FF
:10095800F800E493F50812279A122CD4900789E03E
:10096800900026F090078AE0900027F090078BE02F
:10097800900028F090078CE0900029F090078DE017
:10098800F56690078EE0F56890078FE0F5699007A7
:1009980090E0F56A900791E0F565900792E0F567B9
:1009A800900793E0F564900794E0F563900795E06D
:1009B80090002AF0900796E090002BF0900797E0BF
:1009C80090002CF0900798E0900041F0900799E093
:1009D800900042F090079AE0900043F090079BE067
:1009E800900044F090079CE0900045F090079DE04F
:1009F800900046F090079EE0900047F090079FE037
:100A0800900048F09007A0E0900033F09007A1E034
:100A1800900034F09007A2E0900035F09007A3E032
:100A2800900036F07400900082F090013AE0700C6B
:100A380090013BE0700690013CE060028004C20A2D
:100A48008002D20A90F807E493900021F0900021E8
:100A5800E0440A900021F0900021E054FE9000212B
:100A6800F07406900012F07402900013F090F802EF
:100A7800E493900014F07403900015F07403900050
:100A880016F07401900017F07405900018F09000AB
:100A980014E0B404067404900018F0900014E0B454
:100AA80003067403900018F07405900019F090F88C
:100AB80004E49390001DF0740090001EF090F80577
:100AC800E49390001FF090F806E493900020F074EF
:100AD800FF900022F0744C900125F0746590012677
:100AE800F07478900127F07475900128F074739071
:100AF8000129F0742090012AF0744190012BF074C0
:100B08003390012CF0743490012DF0743390012E41
:100B1800F0742090012FF07434900130F0745390E9
:100B28000131F07450900132F07444900133F09028
:100B3800007AE0D394014006740090007AF075586A
:100B480001755901740390004CF01200C91204BBDE
:100B5800900014E0B404051206478011900014E0D8
:100B6800D394044005120579800312071512268FC5
:100B7800E5B554FEF5B5900025E4F0900786E4F05D
:100B8800A3F0752400752300754800752A0075299F
:100B980000754900753200753100754A00755400BA
:100BA800755500755A0075510475520175343C75B8
:100BB8003300757000756F007571CD7556007557E7
:100BC80000754300754400754500754600755B0067
:100BD800754700754200754100900006E4F0A3F0E7
:100BE800900008E4F0A3F0755E00755F0090000EB9
:100BF80074FDF0A374E8F0900023E4F074649000AE
:100C080024F0C200D201C202D203754D00756D00F6
:100C1800C294C293C287C290C291C20C7E017F0067
:100C2800900028E0124094900027E02FFF50010E1A
:100C380090000AEEF0A3EFF0900026E0700674FF33
:100C4800900026F090000AE0FEA3E0FFEFD394FFA7
:100C5800EE940F400790000AE4F0A3F074009000AF
:100C680071F07400900079F07400900082F07400C4
:100C780090008DF074009000B4F0E567700375671C
:100C880004743A90074EF074FD90074FF09003D427
:100C9800E0900414F0D2B0D2B7D2A7D2A6D2B1D283
:100CA800A3C207A2B6B39204A2B3B39205D29CD250
:100CB800EC75CF01A298B34005C298123038E513FD
:100CC8006006A299B3B340028005C2991235A8E51F
:100CD8001464016005E514B4040280D5E54DD3948D
:100CE80005400CE55AC394C85002055A754D00E5F5
:100CF80071C394F0501A786F12003FAE6FAF70EF67
:100D0800D394E8EE940340080571757000756F0080
:100D1800C28E7E047F00E54C124094E58D75F00488
:100D2800A4FDACF0EF2DFDEE3CFCE58B75F04084A6
:100D3800FF7E00ED2FFFEC3EFE8E258F26D28EA281
:100D4800B6300401B35003020E8CA2B6300401B3CE
:100D58005003020E8CA2B640670554A20D400575DB
:100D6800FFA0D20DE5B54401F5B5900024E4F0E507
:100D780054D3956640487C837DC2AE25AF26123F8A
:100D8800348E238F24E5482FFF50010E7401124042
:100D9800868E238F24852448755401C28E758D0054
:100DA800758B00754C00D28E7403BE00039F5006ED
:100DB8009000257401F0E543B40603754300D2049E
:100DC800A2B6B35003020E8CC20490006BE0601808
:100DD8001236E9A200B34008E5B54408F5B5800627
:100DE800E5B554F7F5B58002C20090006EE06018D2
:100DF80012383EA202B34008E5B54402F5B58006B4
:100E0800E5B554FDF5B58006E5B554FDF5B5A20781
:100E1800B34004D2878002C287900059E06004D2B0
:100E2800908002C29090004AE0B40104D2948002FB
:100E3800C294900049E0B40104D2938002C293A204
:100E480009B34004D2918002C291900018E0FE904C
:100E58000014E0C39E4009900014E0D394084009B0
:100E680074FB900023F012047290001DE06015904E
:100E7800001DE0FE900017E06E600974FE900023EC
:100E8800F0120472C2CA7E017F00E54E124094E55A
:100E9800CD2FFF50010E8E278F28D2CAE565B401E9
:100EA8004890000EE0FCA3E0FDEFC39DEE9C4039A6
:100EB800B208E52A45296013A208B34008E5B544FD
:100EC80004F5B58006E5B554FBF5B590000EE0FED7
:100ED800A3E0FF900010E0FCA3E0FDEF2DFDEE3C49
:100EE800FC90000EECF0A3EDF0A2B3300501B35076
:100EF80003020FDAA2B3300501B35003020FDAA2DE
:100F0800B35003020FD30555A20D400575FFA0D2BB
:100F18000DE5B54401F5B5900024E4F0E555D39509
:100F2800685003020FD17CEA7D60AE27AF28123FDC
:100F3800348E298F2AE56912409474FF8E048F0538
:100F4800FF1240768C298D2AE5492DFD50010C743D
:100F5800018C068D071240868E298F2A852A49A280
:100F680009B340157464124094900067E08E048FB2
:100F780005FF1240768C298D2A75550190000EE0E8
:100F8800FEA3E0FFAC27AD2812000390000EEEF0A0
:100F9800A3EFF0E567FF124076740AFF12407690DF
:100FA800007BE08C068D0712409474148E048F0524
:100FB800FF124076900010ECF0A3EDF0C2CA75CD98
:100FC8000075CC00754E00D2CAD205A2B3B3400258
:100FD800C205900025E0B40107E556C39406400316
:100FE8000215EEE56D902642F8282873900059E026
:100FF800C394024003021148E551D39401500302FF
:101008001148E55175F040A4FFAEF09003121200AC
:101018001EE0C395455018E55175F040A4FFAEF0A9
:1010280090031112001EE0F52E752D00021148E5FF
:101038005175F040A4FFAEF090031012001EE0C3FB
:10104800954540030210E4E55175F040A4FFAEF069
:1010580090031112001EE55175F040A4FFAEF0E0B8
:10106800FC90030F12001EECFEE0FFEEC39FFEE5AE
:10107800518E0475F040A4FFAEF090031012001ECC
:10108800E0F40425458C0088F0A4FFAEF0E5518F0C
:10109800048E0575F040A4FFAEF090031212001EF6
:1010A800E55175F040A4FFAEF0E0FA90031012008D
:1010B8001EEAFEE0FFEEC39FFECDCCCD8E071240A8
:1010C80076E55175F040A4FFAEF090030F12001EB4
:1010D800E02DFD50010C8C2D8D2E8064E55175F0AE
:1010E80040A4FFAEF090030F12001EE55175F040CA
:1010F800A4FFAEF0E0FC90030E12001EECFEE0FF31
:10110800EEC39F8545F0A4FFAEF0E5518F048E0530
:1011180075F040A4FFAEF090031012001EE0FECD63
:10112800CCCD8E07124076E55175F040A4FFAEF0A5
:1011380090030E12001EE02DFD50010C8C2D8D2EFB
:10114800756D010215EE900059E0C3940240030248
:1011580012FC90004FE0D3955150030212A4E551C0
:1011680075F040A4FFAEF090031812001EE0C3957E
:10117800455018E55175F040A4FFAEF090031712E2
:10118800001EE0F52C752B000212A4E55175F04005
:10119800A4FFAEF090031612001EE0C3954540036D
:1011A800021240E55175F040A4FFAEF0900317120B
:1011B800001EE55175F040A4FFAEF0E0FC90031569
:1011C80012001EECFEE0FFEEC39FFEE5518E047593
:1011D800F040A4FFAEF090031612001EE0F40425C0
:1011E800458C0088F0A4FFAEF0E5518F048E05759C
:1011F800F040A4FFAEF090031812001EE55175F000
:1012080040A4FFAEF0E0FA90031612001EEAFEE0DA
:10121800FFEEC39FFECDCCCD8E07124076E551750B
:10122800F040A4FFAEF090031512001EE02DFD5013
:10123800010C8C2B8D2C8064E55175F040A4FFAE19
:10124800F090031512001EE55175F040A4FFAEF0B2
:10125800E0FC90031412001EECFEE0FFEEC39F8535
:1012680045F0A4FFAEF0E5518F048E0575F040A45B
:10127800FFAEF090031612001EE0FECDCCCD8E0717
:10128800124076E55175F040A4FFAEF090031412B9
:10129800001EE02DFD50010C8C2B8D2CE551B40166
:1012A80023E560D39401401CE55604D395514014BE
:1012B800E545C39405500D90035FE0A829B80006E2
:1012C800952A40028003755102E551B560229000CD
:1012D8004FE0D395514019E55175F040A4FFAEF0A9
:1012E80090031712001EE0A823B8000695244002B8
:1012F80080020560756D020215EE900059E0B40297
:101308002AE55175F040A4FFAEF090031712001EB5
:10131800E0F52C752B00E55175F040A4FFAEF09078
:10132800030E12001EE0F52E752D00900059E0B452
:10133800030F900051E0F52C752B00752E00752DCC
:1013480000756D030215EEE55175F040A4FFAEF08F
:1013580090032012001EE0C3955A40030214249003
:101368000049E07036E551D394014029AE23AF24FB
:10137800AC2DAD2EEDD39FEC9E401AE55175F04093
:10138800A4FFAEF090031E12001EE0A829B80005C5
:10139800D3952A5002800215518034E551D3940226
:1013A8004029AE23AF24AC2DAD2EEDD39FEC9E404B
:1013B8001AE55175F040A4FFAEF090031E12001E0E
:1013C800E0A829B80005D3952A500280021551E5F6
:1013D80051B55237E551C395605030E55604D39561
:1013E800514028AE23AF24AC2BAD2CEFD39DEE9CFF
:1013F8004019E55175F040A4FFAEF090031F1200AC
:101408001EE0A829B80006952A400280020551C2AC
:1014180092E55165526005C207755A00756D040260
:1014280015EEE55175F040A4FFAEF090031A1200D6
:101438001EE0B40117E55175F040A4FFAEF090032B
:101448002012001EE0240AC3955A40030214FA75BC
:101458003064752F00A207B3500B900060E024059C
:10146800C3954540030214FAE55175F040A4FFAE58
:10147800F090031D12001EE0C395454064E55175C8
:10148800F040A4FFAEF090031C12001EE55175F069
:1014980040A4FFAEF0E0FC90031B12001EECFEE03F
:1014A800FFEEC39F8545F0A4FFAEF0E5518F048E93
:1014B8000575F040A4FFAEF090031D12001EE0FE7B
:1014C800CDCCCD8E07124076E55175F040A4FFAE25
:1014D800F090031B12001EE02DFD50010C8C2F8D87
:1014E80030AE23AF24AC2FAD30EFD39DEE9C40023D
:1014F800D207756D050215EEE551B4010990005942
:10150800E0C3940240030215CE900358E0D39545FA
:1015180050030215CE900356E0C395455040900302
:1015280057E0FE900355E0F4042EFE900356E0F4D5
:101538000425458E0088F0A4FFAEF0900358E0FC27
:10154800900356E0F4042C8E048F05FF1240769029
:101558000355E02DFD50010C8C2B8D2C802C900315
:1015680055E0FE900354E0F4042E8545F0A4FFAE48
:10157800F0900356E08E048F05FF124076900354D6
:10158800E02DFD50010C8C2B8D2CE551C39560503E
:1015980030E55604D395514028AE23AF24AC2BAD8B
:1015A8002CEFD39DEE9C4019E55175F040A4FFAE99
:1015B800F090031F12001EE0A829B80006952A40E3
:1015C800028003755102900049E0B40106E55164B8
:1015D8000160028003755102E55165526005C2073A
:0615E800755A00756D004C
:10264200020FF402114E02130202134F02142A0265
:02265200150071
:1015EE00900050E02402A823B80007D395244002AF
:1015FE00C207900025E0B40109900059E0C394039E
:10160E004003021776900049E060030216C5E551CB
:10161E00D394014034E55175F040A4FFAEF0900331
:10162E001412001EE0A823B8001FD39524401AE51B
:10163E005175F040A4FFAEF090031F12001EE0A8FB
:10164E0029B80005D3952A500280021551E551D3D1
:10165E009401402FE55175F040A4FFAEF0900312B7
:10166E0012001EE0C39545501AE55175F040A4FFD7
:10167E00AEF090031E12001EE0A829B80005D39507
:10168E002A500280021551E551D394014022E556AD
:10169E0004C39551501AE55175F040A4FFAEF09079
:1016AE00031E12001EE0A829B80005D3952A500289
:1016BE008002155102176BE551D394024034E55167
:1016CE0075F040A4FFAEF090031412001EE0A823A4
:1016DE00B8001FD39524401AE55175F040A4FFAE13
:1016EE00F090031F12001EE0A829B80005D3952A1A
:1016FE00500280021551E551D39402402FE55175E9
:10170E00F040A4FFAEF090031212001EE0C3954508
:10171E00501AE55175F040A4FFAEF090031E120072
:10172E001EE0A829B80005D3952A50028002155153
:10173E00E551D394024022E55604C39551501AE563
:10174E005175F040A4FFAEF090031E12001EE0A8EB
:10175E0029B80005D3952A500280021551E551652E
:10176E00526005C207755A00900060E0D39545504F
:10177E0009900054E0C395455002C207900059E00D
:10178E0070030219DBA2A5B34008A2A4B340030262
:10179E0019C4AE35AF367441D39F749C9E40057804
:1017AE003512003FAE35AF36EFB48806EEB41302F5
:1017BE0080030219A1A2A55003021864900059E0FB
:1017CE00B4010B90004FE0D395604002056090008D
:1017DE0059E0B40254E55175F040A4FFAEF0900309
:1017EE002012001EE0C3955A503F90004FE0D39553
:1017FE00514021E55604D395514019E55175F040FD
:10180E00A4FFAEF090031412001EE0A823B8000649
:10181E00952440028002055190004FE0F560E5519D
:10182E0065526005C207755A00900059E0B4032650
:10183E0090004FE0D395514008E55604D395515092
:10184E00028002055190004FE0F560E5516552604F
:10185E0005C207755A00A2A450030219A19000599F
:10186E00E0B4016E900049E07035E551D39401402B
:10187E0029E55175F040A4FFAEF090031E12001E34
:10188E00E0A829B8000FD3952A400A1551755A00C1
:10189E00855160800385516080037560018033E55A
:1018AE0051D394024029E55175F040A4FFAEF0905B
:1018BE00031E12001EE0A829B8000FD3952A400A75
:1018CE001551755A008551608003855160800375EE
:1018DE006002900059E0D394015003021995E5512E
:1018EE0075F040A4FFAEF090032012001EE0C395E9
:1018FE005A4003021995900049E07041E551D39486
:10190E00014034E55175F040A4FFAEF09003111282
:10191E00001EE0A823B8001FD39524401AE5517588
:10192E00F040A4FFAEF090031E12001EE0A829B8EE
:10193E000005D3952A500280021551803FE551D300
:10194E0094024034E55175F040A4FFAEF0900311BF
:10195E0012001EE0A823B8001FD39524401AE551AB
:10196E0075F040A4FFAEF090031E12001EE0A829F1
:10197E00B80005D3952A500280021551E5516552E3
:10198E006005C207755A00E556B40704055E80036C
:10199E00755E00E563B4010EAE35AF36EF64407090
:1019AE0005EE649C6002800EA2A54003755801A24C
:1019BE00A44003755802A2A5B3B35006A2A4B3B3B4
:1019CE0040028006753600753500021AC9A2A5B30D
:1019DE004008A2A4B34003021AB5AE35AF36744127
:1019EE00D39F749C9E4005783512003FAE35AF36BE
:1019FE00EFB48806EEB413028003021AB5A2A54016
:101A0E006F900068E0605A90004AE0B401079000C1
:101A1E004AE4F0800690004A7401F090004AE070AB
:101A2E0005756003800375600490004AE0B40104FC
:101A3E00D2948002C294E551B4041AE55175F04077
:101A4E00A4FFAEF090031E12001EE0A829B80005F8
:101A5E00D3952A50028008755103C207755A00802B
:101A6E0003756004E556B40704055E8003755E00D9
:101A7E00A2A44033900069E06021900049E0B401D7
:101A8E0007900049E4F080069000497401F0900040
:101A9E0049E0B40104D2938002C293E556B4070420
:101AAE00055E8003755E00A2A5B3B35006A2A4B373
:101ABE00B340028006753600753500E558655960ED
:101ACE0006900082E06003021C51C29C75140075E2
:101ADE001300C2CAE558902654F8282873801212B3
:101AEE002CD4800D122DAD8008122E868003122F5D
:011AFE005F88
:0F265400021AEB021AED021AF2021AF7021AFC2E
:101AFF00900029E090007AF0E566900057F0E568D5
:101B0F00900062F0E569900063F0E56A900074F070
:101B1F00E56590007CF0E56790007DF0E56490004E
:101B2F0080F0E563900081F090002AE090013AF098
:101B3F0090002BE090013BF090002CE090013CF0E6
:101B4F00900041E0900090F0900042E0900091F002
:101B5F00900043E0900092F0900044E0900093F0EA
:101B6F00900045E0900094F0900046E0900095F0D2
:101B7F00900047E0900096F0900048E0900097F0BA
:101B8F00900033E0900099F0900034E090009AF0CC
:101B9F00900035E090009BF0900036E090009CF0B4
:101BAF007400900082F0744C900125F074659001E0
:101BBF0026F07478900127F07475900128F07473F3
:101BCF00900129F0742090012AF0744190012BF0BC
:101BDF00743390012CF0743490012DF07433900114
:101BEF002EF0742090012FF07434900130F0745364
:101BFF00900131F07450900132F07444900133F041
:101C0F009003D4E0900414F0743A90074EF074FDF2
:101C1F0090074FF01200C9900004E4F0A3F0900079
:101C2F00067475F0A37430F09000087475F0A37407
:101C3F0030F0855859D2CA754C00D29C741B900055
:101C4F0023F0E556C394065005E551B55202804E78
:101C5F00C207E55175F040A4FFAEF09003221200C9
:101C6F001EE030E003D38001C39296E55175F0403A
:101C7F00A4FFAEF090032312001EE030E003D380E8
:101C8F0001C39295855152AE29AF2A7405BE000348
:101C9F009F5007E545D3940550028002D292E55636
:101CAF00D394055003021D76C207E551D39401402A
:101CBF0059E55175F040A4FFAEF090031E12001EBF
:101CCF00E0A829B80007D3952A40021551E55165C0
:101CDF00526035E55175F040A4FFAEF0900322122B
:101CEF00001EE030E003D38001C39296E55175F0FA
:101CFF0040A4FFAEF090032312001EE030E003D3A8
:101D0F008001C39295855152805DE556B4061A90B5
:101D1F0000ACE030E003D38001C392969000ADE0B9
:101D2F0030E003D38001C39295E556B4071A9000B3
:101D3F00A5E030E003D38001C392969000A6E03077
:101D4F00E003D38001C39295E556B4081A90009E24
:101D5F00E030E003D38001C3929690009FE030E023
:101D6F0003D38001C39295900072E06058E54575EA
:101D7F00F00284FF7E0090014E12001EE0F55CE53C
:101D8F004775F00A84FF7E0090024E12001EE0F5A8
:101D9F005DE55C255DD39464400BE55C255DC394E4
:101DAF0064F55C8003755C00E55C75F00284FF7E72
:101DBF00008F5CEFC394335007EF24CDF55C8003A5
:101DCF00755CFF801CE54575F00284FF7E00900175
:101DDF004E12001EE075F00284FF7E00EF24CDF559
:101DEF005CE595C3955C4004C2A28002D2A2A20713
:101DFF00B34005E556B407037571CDE595C39571ED
:101E0F004004C2A18002D2A1E543C394064003025D
:101E1F00241AA2EDB3500302241AC2EDE543600366
:101E2F00021F7C7E017F00E5BE124094E5BD2FFFAF
:101E3F0050010E900000EEF0A3EFF0900029E0B4F7
:101E4F0001177E0F7FFF900000E0FCA3E0FD120062
:101E5F0003900000EEF0A3EFF0900079E0B4025B86
:101E6F00900000E0FEA3E0FF90000AE0FCA3E0FD7D
:101E7F00EDD39FEC9E400F900000E0F8A3E09000A0
:101E8F000AC8F0A3C8F0900000E0FEA3E0FF9000A6
:101E9F000CE0FCA3E0FDEFD39DEE9C400F90000003
:101EAF00E0F8A3E090000CC8F0A3C8F0900000E0A9
:101EBF00FEA3E0FF74041240868F44900079E07017
:101ECF0060900000E0FEA3E0FF90000AE0FCA3E0BA
:101EDF00FDEFD39DEE9C400D120003900000EEF03D
:101EEF00A3EFF08007900000E4F0A3F0900000E073
:101EFF00FEA3E0FF7410124094900026E08E048F32
:101F0F0005FF124076900000ECF0A3EDF07400D3C3
:101F1F009D74019C4008900001E0F54480037544D6
:101F2F00FFE54475F00AA4FFAEF074198E048F0517
:101F3F00FF1240768D45ED2532FFAE3150010E7404
:101F4F00011240868F45854532753100EFD394627B
:101F5F004003754562900072E06401600690006670
:101F6F00E060028005754301800375BB17E543B43C
:101F7F000102800302206C7E017F00E5BE124094B7
:101F8F00E5BD2FFF50010E900000EEF0A3EFF09093
:101F9F000072E0B4017EE53445336025AC33AD34D7
:101FAF001DBDFF011C8F028E038C068D07903D34E3
:101FBF0012002EE493FE740193FFEFC39AEE9B4041
:101FCF0002800578331240BEAE33AF3474B3BE0017
:101FDF0025D39F4021900000E0FCA3E0FD0FBF0040
:101FEF00010E903D3412002EE493FE740193FFED29
:101FFF00C39FEC9E40028005783312003FAE33AF93
:10200F0034E56A12409474648E048F05FF12407693
:10201F008D478033900066E0602D900000E0FEA3B6
:10202F00E0FFEFD39400EE9408400F900066E0B409
:10203F000104C2098002D209800D900066E0B4014C
:10204F0004D2098002C209900072E0640260069017
:10205F000066E0600575BB168003754302E543B467
:10206F000202800302215A7E017F00E5BE124094D6
:10207F00E5BD2FFF50010E900000EEF0A3EFF090A2
:10208F000072E0B4027EE53445336025AC33AD34E5
:10209F001DBDFF011C8F028E038C068D07903BCA5E
:1020AF0012002EE493FE740193FFEFC39AEE9B4050
:1020BF0002800578331240BEAE33AF3474B3BE0026
:1020CF0025D39F4021900000E0FCA3E0FD0FBF004F
:1020DF00010E903BCA12002EE493FE740193FFEDA4
:1020EF00C39FEC9E40028005783312003FAE33AFA2
:1020FF0034E56A12409474648E048F05FF124076A3
:10210F008D478033900066E0602D900000E0FEA3C5
:10211F00E0FFEFD39400EE9408400F900066E0B418
:10212F000104C2098002D209800D900066E0B4015B
:10213F0004D2098002C209900072E0700375470053
:10214F00900066E07002C20975BB1FE543B40345FA
:10215F007E017F00E5BE124094E5BD2FFF50010EBA
:10216F00900000EEF0A3EFF0740912409474E68E25
:10217F00048F05FF1240768C418D42E54A2DFD50AC
:10218F00010C74018C068D071240868E418F42859B
:10219F00424A75BB19E543B4040280030223027E51
:1021AF00017F00E5BE124094E5BD2FFF50010E9058
:1021BF000000EEF0A3EFF074041240868F4BE5643D
:1021CF00B40102800302228F756B00756B00E56B03
:1021DF00D39407400302227CE56B9000411240AC80
:1021EF00E0D3954B501AE56B9000411240ACE0F4F0
:1021FF0004254BFEE56B9000371240ACEEF08017D4
:10220F00E56B9000411240ACE0C3954BFEE56B903F
:10221F0000371240ACEEF0E56BC394044009900018
:10222F0084E0C3956B503BE56B6029E56B900037FD
:10223F001240ACFEE0FFEE90003FE0D39F4013E56D
:10224F006B9000371240ACE090003FF0E56B9000D0
:10225F0040F0800E900037E090003FF07400900047
:10226F0040F0786B740126F640030221DD900040A8
:10227F00E0F4042408F556E556D394054002C292C3
:10228F00E564D39401402FE54BD3946E4004D20EF6
:10229F008002C20E755605E564B40205A20EB34066
:1022AF00028003755607E564B40306A20EB3B3406C
:1022BF00028003755607E55765566008E55104F52A
:1022CF0052855657E556B40708E5B54480F5B580F5
:1022DF0006E5B5547FF5B5E55664066005E556B4D9
:1022EF000808E5B54410F5B58006E5B554EFF5B52A
:1022FF0075BB13E543B4050280030224167E017FEC
:10230F0000E5BE124094E5BD2FFF50010E90000076
:10231F00EEF0A3EFF074041240868F46E563B4022B
:10232F00028003022413756B00756B00E56BD39469
:10233F000340030223CAE56B9000331240ACE0D395
:10234F009546501AE56B9000331240ACE0F404252B
:10235F0046FEE56B90002D1240ACEEF08017E56B5A
:10236F009000331240ACE0C39546FEE56B90002D14
:10237F001240ACEEF0E56B6029E56B90002D12403A
:10238F00ACFEE0FFEE900031E0D39F4013E56B9081
:10239F00002D1240ACE0900031F0E56B900032F070
:1023AF00800E90002DE0900031F07400900032F01C
:1023BF00786B740126F6400302233B900082E07095
:1023CF0043E52A45296036E558C39403500A900027
:1023DF0032E004C3940340028007900032E004F51A
:1023EF0058E558D39402400A900032E004D3940287
:1023FF0050028007900032E004F5588007900032B9
:10240F00E004F55875BB180543D2ECE55ED3940490
:10241F00500302250275CF01C2A2AE35AF367488C4
:10242F00D39F74139E4005A2A5B34014AE35AF36AB
:10243F007488D39F74139E4005A2A4B340028048B2
:10244F00783512003FAE35AF36EFB4883BEEB4139C
:10245F0037A2A5B3500990004FE0D3955150028099
:10246F000405518011A2A5B3500890004FE06551AB
:10247F0060028002D207A2A4B35007E551D39401A2
:10248F00500280041551C207A2A5B3B35006A2A4EF
:10249F00B3B340028006753600753500E5516552BD
:1024AF006035E55175F040A4FFAEF09003221200A5
:1024BF001EE030E003D38001C39296E55175F040E2
:1024CF00A4FFAEF090032312001EE030E003D38090
:1024DF0001C39295855152A20740057571CD8003B6
:1024EF007571FFE595C395714004C2A18002D2A119
:1024FF00022424A20DB3500DAE25AF2674E8C39F5E
:10250F0074039E4002800575FFA0D20DAE25AF2645
:10251F00EFD39420EE944E5003022616120472C28B
:10252F008E758D00758B00754C00D28EC20775703D
:10253F0000756F007571CD755104752400752300FA
:10254F00755400755A00C287900059E06004D2900C
:10255F008002C29090004AE0B40104D2948002C27B
:10256F0094900049E0B40104D2938002C293A2096F
:10257F00B34004D2918002C29190006BE0601812B8
:10258F0036E9A200B34008E5B54408F5B58006E585
:10259F00B554F7F5B58002C20090006EE0601812D6
:1025AF00383EA202B34008E5B54402F5B58006E512
:1025BF00B554FDF5B58006E5B554FDF5B590000EA3
:1025CF0074FDF0A374E8F0E543B40603754300907F
:1025DF000025E4F0752600752500758D00758B00BC
:1025EF00754C00900024E0C394035008900024E041
:1025FF0004F080067403900024F0900024E0B403EC
:10260F0006E5B554FEF5B5AE27AF28EFD39410EE1F
:10261F009427401CC2CA75CD0075CC007528007573
:10262F002700D2CA754E00752A007529007555000E
:03263F00020CB9D1
:1039F00000000100013201640196019602000212EA
:103A000002240200020003000340038003C00400FC
:103A10000440048004C005000600060006000600FD
:103A2000060006000600060000FF01310163019553
:103A300001FF01FF0211022302FF02FF02FF033F09
:103A4000037F03BF03FF043F047F04BF04FF05FFA0
:103A500006FF06FF06FF06FF06FF06FF06FF06FF3E
:103A60000FAA0FA50F9F0F9A0F940F8D0F870F802E
:103A70000F780F710F680F600F570F4E0F450F3BF8
:103A80000F300F250F1A0F0E0F020EF50EE80EDB8A
:103A90000ECC0EBE0EAE0E9F0E8E0E7D0E6C0E5A0E
:103AA0000E470E340E200E0C0DF70DE20DCB0DB5AA
:103AB0000D9D0D850D6D0D540D3A0D200D050CE974
:103AC0000CCE0CB10C940C760C580C3A0C1B0BFB66
:103AD0000BDB0BBB0B9A0B790B570B350B130AF156
:103AE0000ACE0AAB0A870A640A400A1C09F809D4FC
:103AF00009B0098C09670943091F08FB08D608B2F9
:103B0000088E086A0846082307FF07DC07B90796EE
:103B100007730751072F070D06EC06CA06AA068988
:103B200006690649062A060A05EC05CD05B0059288
:103B300005750558053C0520050504EA04CF04B5C4
:103B4000049C04820469045104390422040B03F424
:103B500003DE03C803B2039D038903750361034DAC
:103B6000033B03280316030402F202E102D102C060
:103B700002B002A00291028202730265025702495A
:103B8000023C022F02220216020901FD01F201E6A7
:103B900001DB01D001C601BB01B101A7019D019468
:103BA000018B0182017901700168016001580150A7
:103BB0000148014101390132012B0125011E011883
:103BC0000111010B010500FF00FA0FA60FA00F99CC
:103BD0000F920F8B0F840F7C0F740F6B0F620F58B7
:103BE0000F4E0F430F380F2C0F1F0F120F050EF73C
:103BF0000EE80ED80EC80EB70EA50E930E800E6CF2
:103C00000E580E420E2C0E150DFD0DE40DCB0DB110
:103C10000D950D790D5D0D3F0D200D010CE10CC0D2
:103C20000C9E0C7C0C590C350C100BEA0BC40B9E33
:103C30000B760B4F0B260AFD0AD40AAA0A800A55F6
:103C40000A2A09FF09D409A8097C0950092508F99D
:103C500008CD08A10875084A081E07F307C8079D84
:103C600007730749072006F706CE06A6067E065705
:103C70000630060A05E405BF059B057705540532A5
:103C8000051004EF04CE04AE048F04710453043510
:103C9000041903FD03E203C703AD0394037B03632D
:103CA000034B0334031E030802F302DE02CA02B60A
:103CB00002A30291027F026D025C024C023C022CC4
:103CC000021D020E020001F201E401D701CA01BE89
:103CD00001B101A6019A018F0185017A0170016687
:103CE000015D0153014A01410139013101290121DD
:103CF00001190112010B010400FD00F700F000EAB8
:103D000000E400DE00D900D300CE00C900C400BF2B
:103D100000BA00B500B100AD00A800A400A0009C4E
:103D2000009900950091008E008A00870084008130
:043D3000007E007B96
:10266300751A00751900AE19AF1AAC17AD18EDC382
:102673009FEC9E401674FF12406675CF01781A7462
:102683000126F6500418E436F650DB22900786E460
:10269300F0A3F0751000750F00751300751400C2D8
:1026A3000FD21022C2AF75D900758F0375B7A57508
:1026B300B7F190F800E4F0758F0175B7A575B7F120
:1026C300E50890F800F075B7A575B7F190F801E447
:1026D300F075B7A575B7F190079DE090F802F07516
:1026E300B7A575B7F19007A1E090F803F075B7A50A
:1026F30075B7F190079EE090F804F075B7A575B72C
:10270300F190079FE090F805F075B7A575B7F190C4
:1027130007A0E090F806F075B7A575B7F19007A28A
:10272300E090F807F0758F0075D940D2AF2290077B
:1027330088E0B4AB61C2AF75D90075B62275F522D6
:10274300758F0375B7A575B7F1740090F600F07532
:102753008F01750A00750900AE09AF0A7413BE0034
:10276300279F402475B7A575B7F190078912001EFE
:10277300E0FC90F60012001EECF0780A740126F6D5
:10278300500418E436F650D0758F0075F51175B600
:102793002075D940D2AF22C2AF75D90075F5227525
:1027A3000A00750900AE09AF0A7413BE00229F40E8
:1027B3001F90F60012001EE493FC90078912001E7E
:1027C300ECF0780A740126F6500418E436F650D576
:1027D30075F51175D940D2AF22900788E0B4AA02EB
:1027E3008003022919C2AF75D90075B62275F52287
:1027F300758F0375B7A575B7F1740090EE00F0758A
:10280300B7A575B7F1740090F000F075B7A575B76B
:10281300F1740090F200F075B7A575B7F1740090EC
:10282300F400F0758F01750A00750900AE09AF0A4F
:1028330074FFC39F74019E402475B7A575B7F190CB
:10284300004E12001EE0FC90EE0012001EECF07829
:102853000A740126F6500418E436F650CF750A00C0
:10286300750900AE09AF0A74FFC39F74019E40242B
:1028730075B7A575B7F190024E12001EE0FC90F0FB
:102883000012001EECF0780A740126F6500418E4D6
:1028930036F650CF750A00750900AE09AF0A74FF0A
:1028A300C39F74019E402475B7A575B7F190044E7C
:1028B30012001EE0FC90F20012001EECF0780A7485
:1028C3000126F6500418E436F650CF750A00750950
:1028D30000AE09AF0A74FFC39F74019E402475B70D
:1028E300A575B7F190064E12001EE0FC90F400129D
:1028F300001EECF0780A740126F6500418E436F64C
:1029030050CF758F0075F51175B62075D940D2AFCC
:10291300743A90074EF022900788E0B4AA0280032D
:10292300022A57C2AF75D90075B62275F522758F85
:102933000375B7A575B7F1740090E600F075B7A5F8
:1029430075B7F1740090E800F075B7A575B7F17429
:102953000090EA00F075B7A575B7F1740090EC002C
:10296300F0758F01750A00750900AE09AF0A74FF8F
:10297300C39F74019E402475B7A575B7F190004EAF
:1029830012001EE0FC90E60012001EECF0780A74C0
:102993000126F6500418E436F650CF750A0075097F
:1029A30000AE09AF0A74FFC39F74019E402475B73C
:1029B300A575B7F190024E12001EE0FC90E80012DC
:1029C300001EECF0780A740126F6500418E436F67B
:1029D30050CF750A00750900AE09AF0A74FFC39F93
:1029E30074019E402475B7A575B7F190044E12008B
:1029F3001EE0FC90EA0012001EECF0780A74012637
:102A0300F6500418E436F650CF750A00750900AE87
:102A130009AF0A74FFC39F74019E402475B7A5755F
:102A2300B7F190064E12001EE0FC90EC0012001E5F
:102A3300ECF0780A740126F6500418E436F650CF09
:102A4300758F0075F51175B62075D940D2AF743AFC
:102A530090074EF022900788E0B4AA028003022B6D
:102A630095C2AF75D90075B62275F522758F0375BA
:102A7300B7A575B7F1740090DE00F075B7A575B70B
:102A8300F1740090E000F075B7A575B7F17400908C
:102A9300E200F075B7A575B7F1740090E400F07526
:102AA3008F01750A00750900AE09AF0A74FFC39F51
:102AB30074019E402475B7A575B7F190004E1200BE
:102AC3001EE0FC90DE0012001EECF0780A74012672
:102AD300F6500418E436F650CF750A00750900AEB7
:102AE30009AF0A74FFC39F74019E402475B7A5758F
:102AF300B7F190024E12001EE0FC90E00012001E9F
:102B0300ECF0780A740126F6500418E436F650CF38
:102B1300750A00750900AE09AF0A74FFC39F7401FB
:102B23009E402475B7A575B7F190044E12001EE0C0
:102B3300FC90E20012001EECF0780A740126F650B5
:102B43000418E436F650CF750A00750900AE09AFD4
:102B53000A74FFC39F74019E402475B7A575B7F12E
:102B630090064E12001EE0FC90E40012001EECF0F2
:102B7300780A740126F6500418E436F650CF758FA0
:102B83000075F51175B62075D940D2AF743A900728
:102B93004EF022900788E0B4AA028003022CD3C22D
:102BA300AF75D90075B62275F522758F0375B7A574
:102BB30075B7F1740090D600F075B7A575B7F174C9
:102BC3000090D800F075B7A575B7F1740090DA00DE
:102BD300F075B7A575B7F1740090DC00F0758F013F
:102BE300750A00750900AE09AF0A74FFC39F74012B
:102BF3009E402475B7A575B7F190004E12001EE0F4
:102C0300FC90D60012001EECF0780A740126F650F0
:102C13000418E436F650CF750A00750900AE09AF03
:102C23000A74FFC39F74019E402475B7A575B7F15D
:102C330090024E12001EE0FC90D80012001EECF031
:102C4300780A740126F6500418E436F650CF750A54
:102C530000750900AE09AF0A74FFC39F74019E405B
:102C63002475B7A575B7F190044E12001EE0FC90D1
:102C7300DA0012001EECF0780A740126F6500418EC
:102C8300E436F650CF750A00750900AE09AF0A7431
:102C9300FFC39F74019E402475B7A575B7F19006D5
:102CA3004E12001EE0FC90DC0012001EECF0780ACD
:102CB300740126F6500418E436F650CF758F00756C
:102CC300F51175B62075D940D2AF743A90074EF01E
:102CD30022C2AF75D90075F522750A00750900AED9
:102CE30009AF0A74FFC39F74019E401F90EE001248
:102CF300001EE493FC90004E12001EECF0780A7460
:102D03000126F6500418E436F650D4750A00750906
:102D130000AE09AF0A74FFC39F74019E401F90F079
:102D23000012001EE493FC90024E12001EECF07899
:102D33000A740126F6500418E436F650D4750A00D6
:102D4300750900AE09AF0A74FFC39F74019E401F4B
:102D530090F20012001EE493FC90044E12001EEC4D
:102D6300F0780A740126F6500418E436F650D47548
:102D73000A00750900AE09AF0A74FFC39F74019E70
:102D8300401F90F40012001EE493FC90064E1200C4
:102D93001EECF0780A740126F6500418E436F65057
:102DA300D475F51175D940D2AF22C2AF75D900756C
:102DB300F522750A00750900AE09AF0A74FFC39FB7
:102DC30074019E401F90E60012001EE493FC9000E5
:102DD3004E12001EECF0780A740126F6500418E433
:102DE30036F650D4750A00750900AE09AF0A74FFB0
:102DF300C39F74019E401F90E80012001EE493FCE1
:102E030090024E12001EECF0780A740126F650046C
:102E130018E436F650D4750A00750900AE09AF0AF6
:102E230074FFC39F74019E401F90EA0012001EE4CA
:102E330093FC90044E12001EECF0780A740126F6FF
:102E4300500418E436F650D4750A00750900AE092B
:102E5300AF0A74FFC39F74019E401F90EC001200E1
:102E63001EE493FC90064E12001EECF0780A7401E7
:102E730026F6500418E436F650D475F51175D9408A
:102E8300D2AF22C2AF75D90075F522750A00750954
:102E930000AE09AF0A74FFC39F74019E401F90DE0A
:102EA3000012001EE493FC90004E12001EECF0781A
:102EB3000A740126F6500418E436F650D4750A0055
:102EC300750900AE09AF0A74FFC39F74019E401FCA
:102ED30090E00012001EE493FC90024E12001EECE0
:102EE300F0780A740126F6500418E436F650D475C7
:102EF3000A00750900AE09AF0A74FFC39F74019EEF
:102F0300401F90E20012001EE493FC90044E120056
:102F13001EECF0780A740126F6500418E436F650D5
:102F2300D4750A00750900AE09AF0A74FFC39F7414
:102F3300019E401F90E40012001EE493FC90064E95
:102F430012001EECF0780A740126F6500418E436D9
:102F5300F650D475F51175D940D2AF22C2AF75D9E9
:102F63000075F522750A00750900AE09AF0A74FFF2
:102F7300C39F74019E401F90D60012001EE493FC71
:102F830090004E12001EECF0780A740126F65004ED
:102F930018E436F650D4750A00750900AE09AF0A75
:102FA30074FFC39F74019E401F90D80012001EE45B
:102FB30093FC90024E12001EECF0780A740126F680
:102FC300500418E436F650D4750A00750900AE09AA
:102FD300AF0A74FFC39F74019E401F90DA00120072
:102FE3001EE493FC90044E12001EECF0780A740168
:102FF30026F6500418E436F650D4750A0075090015
:10300300AE09AF0A74FFC39F74019E401F90DC009A
:1030130012001EE493FC90064E12001EECF0780A98
:10302300740126F6500418E436F650D475F511757C
:10303300D940D2AF22E51464046006E59964FF60C9
:10304300028031A20F4004D20F8027E51460087478
:10305300E62514900023F0E513600874F02513901F
:103063000023F0E514B4010280FE7514007513000B
:10307300C20F8002C20FE514903993F828287375A4
:103083001400E599B4FF03751301E599B4FE0375C4
:103093001302E599B4FD03751303E599B4FC0375B5
:1030A3001304E599B4FA03751305E599B4FB0675A2
:1030B3001401120472E599B4F9067514041204722A
:1030C300E599D394E54007E599C394F0400280164F
:1030D3008599157514027E017F00E515C394E612E8
:1030E30040948E0D8F0E900786E4F0A3F0E599D3FC
:1030F30094C44007E599C394E64002802885991556
:1031030075140374E5C39515F50E750D00AE0DAF7B
:103113000E9039F012002EE493F874019390078611
:10312300C8F0A3C8F0D2990235A7900786E0FEA3A2
:10313300E0FFEFC39400EE94054009EFD394FFEE54
:1031430094064013900786E0FEA3E0FF90004E1222
:10315300001EE599F0800385996C90078612000E96
:10316300900786E0FEA3E0FFEFB40106EEB407028A
:1031730080030233B790074EE0B43C02800302336E
:10318300B7A20AB35005A20BB340030232AAC29CF2
:1031930090007AE090078CF0900057E090078DF054
:1031A300900062E090078EF0900063E090078FF04C
:1031B300900074E0900790F090007CE0900791F00D
:1031C30090007DE0900792F0900080E0900793F0EC
:1031D300900081E0900794F090013AE0900795F019
:1031E30090013BE0900796F090013CE0900797F048
:1031F300900090E0900798F0900091E0900799F08C
:10320300900092E090079AF0900093E090079BF073
:10321300900094E090079CF0900095E090079DF05B
:10322300900096E090079EF0900097E090079FF043
:10323300900099E09007A0F090009AE09007A1F029
:1032430090009BE09007A2F090009CE09007A3F011
:103253007400900082F01200C974AB900788F012DA
:0A326300273174AA900788F0E5589F
:0639930002308202312D1A
:10326D009039B4F828287380121227DC800D1229AA
:0B327D001A8008122A588003122B96BA
:0F39B40002327402327602327B02328002328596
:10328800900788E4F090013AE0700C90013BE07000
:103298000690013CE060028004C20A8002D20A0261
:1032A80033ACC29C900078E0900789F090005EE013
:1032B80090078AF090005FE090078BF090007AE02A
:1032C80090078CF0900057E090078DF0900062E036
:1032D80090078EF0900063E090078FF0900074E004
:1032E800900790F090007CE0900791F090007DE0CE
:1032F800900792F0900080E0900793F0900081E0B2
:10330800900794F090013AE0900795F090013BE027
:10331800900796F090013CE0900797F0900090E0BD
:10332800900798F0900091E0900799F0900092E053
:1033380090079AF0900093E090079BF0900094E03B
:1033480090079CF0900095E090079DF0900096E023
:1033580090079EF0900097E090079FF0900099E00A
:103368009007A0F090009AE09007A1F090009BE0F1
:103378009007A2F090009CE09007A3F074009000E2
:1033880082F074AB900788F012273174AA900788EE
:10339800F01227DC12291A122A58122B96D29C7581
:1033A80099FB80FED29C7514007513007599FB0279
:1033B80035A7900786E0FEA3E0FFEF4E70068599DB
:1033C80010750F00900786E0FEA3E0FF74016F4EB2
:1033D800701BAC0FAD10AA0DAB0EED2BFBEC3AFA3F
:1033E8008A068B0790004E12001EE599F09007861A
:1033F80012000E900786E0FEA3E0FF74026F4E7085
:103408000C1200C98515997514007513000235A7AB
:10341800900786E0FEA3E0FF90004E12001EE5999B
:10342800F090078612000E900786E0FEA3E0FFAC3E
:103438000DAD0E8F028E038C068D07903A28120070
:103448002EE493F9740193FEEAD39EEB9940098523
:1034580015997514007513000235A7900786E0FECC
:10346800A3E0FF90004E12001EE599F09007861227
:10347800000E900786E0FEA3E0FFEFB40006EEB46E
:10348800010280030235A790001CE0D394C7400BCB
:1034980090001CE0C394C8F516801A90001CE0D375
:1034A8009463400B90001CE0C39464F5168006906A
:1034B800001CE0F516E51675F002A4FFAEF08F6B60
:1034C800EF90004E1240ACEFFCE0FDEC9000511282
:1034D80040ACEDFCE0FDEC2DB516028003023599F9
:1034E8000FEF90004E1240ACE56BFFE0FCEF900050
:1034F800521240ACECFFE0FCEFC39CB5160280030F
:10350800023599E56B9000501240ACE56BFFE0FC8A
:10351800EF9000531240ACECFFE0FCEF2CB51671B5
:10352800E56B9000541240ACE0C3951690079DF0EF
:10353800E56B9000551240ACE0C3951690079EF0DD
:10354800E56B9000581240ACE0C3951690079FF0C9
:10355800E56B9000591240ACE0C395169007A0F0B7
:10356800E56B90005A1240ACE0C395169007A1F0A5
:10357800E56B90005B1240ACE0C395169007A2F093
:103588001226A77599F975186475170012266380B5
:0F359800FE7599FF75186475170012266380FE83
:093999000233BA0234180234634F
:1035A70022E5139039A2F82828730236E890078697
:1035B700E0FEA3E0FF90001212001EE0F5999007CD
:1035C7008612000E900786E0FEA3E0FF74116F4E8F
:1035D70070037513000236E88562990236E8900792
:1035E70086E0FEA3E0FF90004E12001EE0F599EF83
:1035F700B40107EEB4070375130090078612000E97
:073607000236E8900787E09E
:0F39A2000235B10235B40235DF0235E502360ACF
:10360E009039C3F82828738524990236DD852A99C6
:10361E000236DD8544990236DD8547990236DD8511
:10362E0051990236DD8560990236DD85569902364E
:10363E00DD8558990236DD756E00900069E07006E2
:10364E00900068E060028016A2A44006E56E440475
:10365E00F56EA2A54006E56E4402F56E801A900046
:10366E004AE0B40106E56E4410F56E900049E0B4F0
:10367E000106E56E4420F56EA207B34006E56E44E2
:10368E0001F56EA209B34006E56E4408F56E856E2F
:10369E0099803CA210B340077599FAC2108017A208
:1036AE000CB3400575990F800B900023E0F59990AF
:1036BE000023E4F0C20C80178542998012854B9945
:0F36CE00800D85469980087599FC80037513005F
:1039C30002361502361B02362102362702362D0235
:1039D300363302363902363F0236450236A1023605
:0D39E300C60236CB0236D00236D50236DAE7
:0B36DD0090078612000E8003120048C8
:0339B1000236E5F6
:1036E8002290006BE0B4010385241190006BE0B4D4
:1036F8000203852A1190006BE0B4030385441190FE
:10370800006BE0B4040385471190006BE0B4050337
:1037180085511190006BE0B4060385561190006B3B
:10372800E0B4070385581190006CE0FE90006DE04E
:10373800C39E50030237BF90006BE0D39404402C23
:1037480090006CE0D39511500990006DE0C395117D
:1037580050028002D20090006CE0D395115009907D
:10376800006DE0C395115002C200804990006BE0E3
:10377800B4041890006DE0C395115002D200900077
:103788006CE0D395114002C200802A90006CE0C31F
:103798009511500990006DE0D3951150028002D226
:1037A8000090006CE0D39511500990006DE0C3952E
:1037B800115002C200807E90006BE0D39404402C2C
:1037C80090006CE0C39511400990006DE0D395110D
:1037D80040028002C20090006CE0C395114009903D
:1037E800006DE0D395114002D200804990006BE053
:1037F800B4041890006CE0C395115002C200900008
:103808006DE0D395114002D200802A90006CE0C38D
:103818009511400990006DE0D395114002D20090B7
:10382800006CE0D39511400990006DE0C3951140FC
:10383800028002C2002290006EE0B40103852411C8
:1038480090006EE0B40203852A1190006EE0B40384
:103858000385441190006EE0B4040385471190007D
:103868006EE0B4050385511190006EE0B40603853F
:10387800561190006EE0B4070385581190006FE070
:10388800FE900070E0C39E500302391490006EE071
:10389800D39404402C90006FE0D395115009900008
:1038A80070E0C3951150028002D20290006FE0D3FD
:1038B80095115009900070E0C395115002C2028022
:1038C8004990006EE0B40418900070E0C395115060
:1038D80002D20290006FE0D395114002C202802A02
:1038E80090006FE0C395115009900070E0D39511D6
:1038F80050028002D20290006FE0D39511500990D7
:103908000070E0C395115002C202807E90006EE004
:10391800D39404402C90006FE0C3951140099000A7
:1039280070E0D3951140028002C20290006FE0C39C
:1039380095114009900070E0D395114002D20280A1
:103948004990006EE0B4041890006FE0C3951150E0
:1039580002C202900070E0D395114002D202802A80
:1039680090006FE0C395114009900070E0D3951165
:103978004002D20290006FE0D39511400990007088
:0B398800E0C3951140028002C2022241
:0940AC002582F5825002058322F1
:10002E00EF2F500205832582F582E5833E2EF58360
:01003E00229F
:08000300C3EF9DFFEE9CFE22FD
:08003F000806B60002180622B3
:0D000E00A3E004F070061240A2E004F0220E
:0840BE000816B6FF02181622D5
:0E408600048007C3CE13CECF13CFD5E0F622B1
:103F3400BC000FBE0008ED8FF084FFADF022E4FE5C
:103F4400FF22BE000DEF60FE54F0606F20E7030215
:103F54003FEAEAC0E0EBC0E078017A0075F001EED8
:103F640020E710EF25E0FFEE33FE0AC5F023C5F08D
:103F740030E7F0EA5407F9096A7A007B0060010827
:103F8400C3EC9E40167004ED9F4010ED9FFDEC9E27
:103F9400FCE5F0CA4ACA03F5F08005E5F003F5F044
:103FA400C3EE13FEEF13FFD9D77908CACBCAD8D012
:103FB400EAFEEBFFD0E0FBD0E0FA22EC8FF084FCC9
:103FC400ED54F045F0C48FF084FEEDC454F045F098
:103FD400C48FF084FDEEC4FE54F02DFFEE540F3C6C
:103FE400FEADF07C0022790078008FF0EC7E082092
:103FF400E70DC3CD33CD33C933C9C833C8DEF0842C
:1040040049F9E5F08FF0BE00E6FD7C00E9FFE8FE2B
:014014002289
:0E409400F88FF0A4FFE5F0CE88F0A42EFE22F7
:10406600600D782B024070007830D8FED5E0F8223B
:10407600EEC0E07E00123F34EFFDEEFCD0E0FE2203
:03000B000240159B
:03001B0002403070
:03002B0002404B45
:030000000240B506
:0940B50075817275D0000207EE5E
:0B001E00E5822FF582E5833EF583228A
:0A40A2000582D582021583158222E3
:10401500C0E0C0F0C083C082C0D075D0001207E3F5
:10402500D0D0D082D083D0F0D0E032C0E0C0F0C094
:1040350083C082C0D075D0001207E6D0D0D082D020
:1040450083D0F0D0E032C0E0C0F0C083C082C0D0E1
:1040550075D0001207E9D0D0D082D083D0F0D0E05F
:014065003228
:00000001FF
